S0160000755461736B657256312E345F424D2E7372656358
S10B8000F02F0020C1BC0000B8
S113801008B5034B03491868402201F01DFD08BD53
S1138020E8F0FF1F38C0000008B5144B1880202862
S11380300ED004D800281CD008281DD119E08028AF
S113804017D080235B00984208D0402814D110E058
S113805061200B49062202F08DF80DE096210622DC
S11380606120C90002F086F8064B1A78064B1A7094
S113807002E0612002F0B8F808BDC046A0F1FF1F7D
S113808070170000E4F0FF1FCCF0FF1F37B5214D3F
S113809021482968402202F00AFC00280FDA1C203B
S11380A02968402202F003FC0024A04209DA28686F
S11380B01A494022802401F0CFFCE40101E080242D
S11380C0240228680378212B04D01449402201F0AB
S11380D0C3FC0024124B29681868402201F0BCFC40
S11380E080231B029C420CD169461C2007310122CB
S11380F002F0DDFB00280BDA022002F0F0FB002482
S113810006E08023DB019C4202D1002000F056FAF5
S1138110201C3EBDE8F0FF1F1C80000038C000009A
S1138120E0F0FF1F054B064A19781170FF22002862
S113813001D1044A12781A707047C046CCF0FF1F70
S1138140C0F0FF1FE4F0FF1F024B1A78024B1A70B5
S11381507047C046C0F0FF1FCCF0FF1F1FB5011CC5
S1138160022368460372184B1B681A7BC272802272
S11381708280D200C280612202731A1C36321278C5
S113818042731A1C3732127882735B6800206A4685
S1138190009301F049FB0D4C2070002810D0002200
S11381A0052101F0A1FA009A520609D508490022D6
S11381B0207801F099FA20788121002201F094FAC4
S11381C0207804B010BDC046E8F0FF1FE4F0FF1FA4
S11381D00404000070B5544CA0B02568867B002DC3
S11381E049D1281C02F024FF402001F009FE4F4B26
S11381F01860402001F004FE4D4B1860281CFFF766
S113820045FF80231B02984201D00123236000F024
S11382109DFB6D20042101F077FF0320FFF79EFFF3
S1138220002800D17EE0434B43481A78434B1A7030
S113823001F066FD424801F063FD01F01BFE051CE0
S113824001F024FE0A21281A01F06BFD3D4801F0DB
S113825057FD01F00FFE8A2101F063FD0BE06B4630
S1138260D8781A7900280ED1D2B2062A0ED0832AE1
S113827001D103F0E7FC301C6946052201F04CFAF9
S11382800028ECD11FE0012807D016E0294B2E4925
S11382901878162201F012FDEDE7D2B2B72A06D003
S11382A0DD2AE8D12368082BE5D12060E3E703F059
S11382B0A7FC264801F024FDDDE792B2301C694694
S11382C001F02AFAD7E7226837231A422AD0194D37
S11382D0287801F031FA002824D028786946402211
S11382E001F01AFA041E1DD06846211C00F02AF978
S11382F0174B68461A88211C002A0FD101F0B0F8E8
S11383000028EAD08020400000F0EAF90228E4D1F5
S113831028781049172201F0D1FCDEE7002201F091
S11383209FF8DAE720B070BDECF0FF1FE8F0FF1F04
S1138330E0F0FF1FE4F0FF1F78C00000CCF0FF1F47
S113834095C00000A4C00000D4C00000ABC0000071
S1138350A0F1FF1FBDC000007047021C0878131C69
S1138360002806D01B78013101329842F6D0002053
S11383700AE000229A56202A06DC00229A56202A75
S113838001D10133F9E7181C704730B50368021CAA
S113839000215956202904D111680133013111609B
S11383A0F6E71D1D0020AB4216D019784CB22F2CD5
S11383B012DDCCB2211C30390001C9B280B20133C4
S11383C0092902D9211C3739C9B20F242140084395
S11383D0116801311160E6E730BD036800229A5646
S11383E0202A05D01A7820218A4301D00133F9E7E5
S11383F000229A56202A01D10133F9E703600020B4
S1138400185643425841704708B5054801F078FCB6
S1138410044801F075FC044801F072FC08BDC04634
S113842064C2000055D0000077C20000F0B52C4AA9
S11384302C4E13780C2253439C59F3181A798BB0A1
S1138440071C019203A820211B225D7901F0FCFA8C
S1138450002F04D0BD4225DD0C34013DFAE722484B
S113846001F04EFC1E4A13780C225343F618B068F0
S113847001F046FC1D4801F043FC13E0206801F0C4
S11384803FFC019B021C30789A421EDB03A90122A7
S113849001F014FC606801F033FC154801F030FC75
S11384A00C34013D002D15D0124E002130784222AB
S11384B001F004FC0028E1D1307840210E4A01F09B
S11384C013F90E4B01201D6007E0019B03A99A1AC2
S11384D092B2DDE7094B281C1D600BB0F0BDC0460D
S11384E0A8F1FF1F9CCD000076C200007AC20000F4
S11384F077C20000CCF0FF1F6D100000F8F0FF1FE2
S113850010B5847B88B0201C6946052201F004F96B
S1138510002813D06946CB780A79012B08D1DD2ACB
S1138520F1D1074B18680028EDD0FFF77FFFEAE789
S113853092B2201C694601F0EFF8E4E708B010BDE0
S1138540F8F0FF1F08B50A1C0349031C0878191C1E
S113855001F0B4FB08BDC046E4F0FF1F154B164AFA
S11385601B6812685868516810B50124884208D104
S1138570D88ED18E884204D1117B1C7B641A611E73
S11385808C4152895B8953402822134201D0022234
S113859014430422134200D01443DA0601D50823FD
S11385A01C430120FFF772FDE30702D50420FFF707
S11385B0D5FD10BDE8F0FF1FE0F0FF1F38B50A4CF1
S11385C0051C21680948402202F050F9012D08D009
S11385D0022002F084F9064B21681868402201F059
S11385E03BFA002038BDC046E8F0FF1F1C800000A5
S11385F0E0F0FF1F08B5044B021C1B68C021D86BB8
S113860001F02CF908BDC046E8F0FF1F7FB505480E
S113861001F076FB01A8FFF7EDFF01A801F070FB64
S113862007B000BD92C200007FB5031C02380B28BE
S113863045D803F03DFC0644114444443A3518251A
S1138640182DFFF7E3FFFFF7DFFE1E4801F058FB8C
S11386501D4B1868213020E01B4B14221868213070
S113866001F0FAF92BE00C3B581E83410420C01A98
S113867001A902F03FFB01A801F042FB13480CE002
S1138680102002F037FB124801F03AFB0C2013E0F3
S11386901020002102F02EFB0E4801F031FB0EE009
S11386A0082002F027FB0C4803E0202002F022FB04
S11386B00A4801F025FB0A200021FFF7B5FF07B0A7
S11386C000BDC046A4C20000E8F0FF1F41C4000082
S11386D0BCC20000CCC20000DCC20000EBC200003F
S11386E0802310B55B0098420BD1164B02241B88E3
S11386F0002B25D1144B1B88002B21D1FFF794FCB0
S113870003E08022104B92001A80104B1A888023B9
S11387105B009A4202D12020FFF786FCFFF776FF28
S1138720FFF772FE0A4801F0EBFA0A4B00241868BE
S1138730213001F0E5FA084B201C1C70FFF776FE8F
S1138740201C10BD9EF1FF1FF6F0FF1FA0F1FF1FBC
S1138750A4C20000E8F0FF1FA8F1FF1F32280FD0C9
S1138760332819D0312824D1134B144A18681268BD
S11387701968134B10401B688B431843800116E0A3
S11387800D4B0E4A1868126819680D4B10401B688F
S11387908B431843C0010AE0074B084A1868126863
S11387A01968074B10401B688B4318430006C00F21
S11387B000E000207047C04654F00F4040F00F40E6
S11387C050F00F40F7B5134F01253B6831201A1CB8
S11387D038321278002400925B8F0193461C40B219
S11387E0F6B2FFF7BBFF002800D02C436D00EDB2BA
S11387F0392E01D0F0B2F1E7FFF7B0FE3B680099E3
S11388001A1C383211705470019A00205A87FFF7ED
S1138810D5FEF7BDE8F0FF1F322807D0332809D072
S113882031280DD1074B1B685B0E06E0054B1B6816
S11388301B0E02E0034B1B68DB090120984300E098
S11388400020704754F00F4038B5031C303B002023
S1138850032B4BD8181C03F02BFB020905078024BB
S1138860A40405E0802403E0002401E080246404DF
S11388705DB264290BD003DC0020612936D003E00B
S1138880692904D06F291AD0012040422EE0184BE8
S1138890E2431968012011401960164B19680A4017
S11388A01A60211C021C03F0E7F8134B1A68012319
S11388B0AB4038321D1C1378AB43137015E00C4BDE
S11388C0211C1A680120A2431A60002203F0D4F884
S11388D0084B1A6814431C60074B1A68012338328A
S11388E01178AB401D1C0D431570002038BDC046E7
S11388F058F00F4054F00F40E8F0FF1F104BC10731
S113890004D51968802292040A4302E019680D4ACA
S11389100A401A601968820703D5802252040A4368
S113892001E0094A0A401A608022410702D5196809
S11389300A4302E0196891430A1C1A607047C04652
S1138940400000F8FFFFFFFDFFFFFFFE0F4B70B577
S11389501B6801211A1C383239331678187801241F
S113896030401870FFF7CAFF30206921264200D03A
S11389706F21451C49B240B26400EDB2FFF764FFB9
S1138980E4B2382D01D0281CEFE770BDE8F0FF1FDA
S11389901E4B10B51A68041C110619D41A689107E5
S11389A018D41A68510717D41A68910616D41A688D
S11389B0510615D41A68910514D41A68510513D4B4
S11389C01A68110512D41B689A0411D5104910E0D5
S11389D010490EE010490CE010490AE0104908E083
S11389E0104906E0104904E0104902E0104900E093
S11389F01049002C04D1081C01F082F9201C04E069
S1138A00201C01F0C1F9001BC0B210BD008004405D
S1138A1088CD000048D000007CCE000040C2000099
S1138A2060C1000027D00000EBC00000A4C100001A
S1138A3020CE00002ECE000038B503F0CDF800247F
S1138A40051C012C03D0022C03D0094802E009487C
S1138A5000E0094801F054F9A54202D1074801F0A9
S1138A604FF90748013401F04BF9032CE9D138BD23
S1138A70FAC2000002C300000BC3000014C30000CC
S1138A8041C40000F0B50C1C93B0161C072801D992
S1138A9000F0A3FC03F016FA08003900B102CE027C
S1138AA0A1042C0388048D04081E05D0042908D1D0
S1138AB00122BD4B00201A70FFF7B8FC051C00F022
S1138AC09DFC02220529F4D003220629F1D00422B8
S1138AD00729EED005220929EBD006220A29E8D07D
S1138AE007220E29E5D008220F29E2D009221029F5
S1138AF0DFD00A221129DCD00025122901D000F090
S1138B007DFCA94B281C1D70D6E70692272901D9A4
S1138B1000F063FC081C03F0D5F928004000D500E0
S1138B206004C300890060046004600460046A0097
S1138B307500C00060046004EC00DC01DC0160042A
S1138B406004600460046004600460046004600401
S1138B50600460046004600460042C00EC00DC0128
S1138B60DC01600452023400380003F06BF800F0BA
S1138B7034FC8E4801F0C4F80020FFF709FF00F030
S1138B802CFCFFF759FF00F028FC101C00F039FF03
S1138B90C0B203F035F800F020FC854801F0B0F8CD
S1138BA0844801F0ADF8844801F0AAF801F06EF9A8
S1138BB00A2101F0B6F8814801F0A2F801F05AF94F
S1138BC00A2101F0AEF808AC7D4801F099F8201CA8
S1138BD001F03AF90A2101F0A4F87A4801F090F87A
S1138BE020880A2101F09DF8774800F0F4FB08A8DA
S1138BF002F04EFA00250570744801F081F808A8C7
S1138C0000F0EDFB1378313B032B01D97048E2E30C
S1138C10704801F075F8069900200856FFF7FCFD2E
S1138C20051E01D16C48DAE36C48D4E31078031CC8
S1138C30313B032B01D96A48CDE340B2FFF7ECFD89
S1138C40051E01D06748C6E3041C01263120471CD9
S1138C5040B2FFB2FFF782FD002801D03443E4B2F2
S1138C607600F6B2352F01D0F8B2F0E7069800F09E
S1138C70ACFEC6B20698013E0123B34001301E1C6F
S1138C80069000F0A2FE012801D1344300E0B44371
S1138C90E0B20021FFF732FEB0E3FFF793FD9CE35F
S1138CA01378313B032BC6D84F4801F029F8069AB4
S1138CB000201056FFF752FD051E01D04B488AE3F1
S1138CC04B488CE3101C079200F07FFE041C07A89D
S1138CD0FFF783FB002801D046487CE3079B2F3431
S1138CE0002160B25956FFF7AFFD002800D174E3AC
S1138CF0F2E70023D356002B02D11021029127E082
S1138D00101C00F062FE3C4B186006A8FFF765FBE0
S1138D10069B1A78002AF0D020218A4352B20421FB
S1138D204C2A02D0572A04D10221344A013311605B
S1138D3005E0422A04D1314A012111605B180693EF
S1138D4006980023C356002BD7D000F05AFE029099
S1138D502B4800F0D5FF08AB20221A705A70029BF2
S1138D60002B00DC39E3244D0C21286800F0D9FFE6
S1138D70244800F0C5FF6A46223210230092039370
S1138D801E4E3268022A45D0042A56D0012A00D049
S1138D9023E3212C38D16F4616372868391C02F09A
S1138DA0E9FC3B7832E0C046A8F1FF1F1EC3000077
S1138DB032C300007DC2000049C30000A4C000000B
S1138DC056C3000068C300006BC300006FC30000FB
S1138DD094C30000A6C30000B9C30000C2C30000CE
S1138DE0CAC30000D9C30000E9C30000F6C30000F1
S1138DF0FAC30000FEC30000A4F1FF1FC8F0FF1F68
S1138E0006C4000017C4000029680B780793079A6A
S1138E10D0B20EE0212C07D16F4616372868391CD2
S1138E2002F0A8FC3B8801E029680B880793079AA5
S1138E3090B23378202119430DE0212C04D1286805
S1138E4007A902F097FC02E02B681B6807933378AC
S1138E5020210798194300F064FF296833685A18E1
S1138E602A60039A0799D21A03920191022B06D021
S1138E70191F48424141182249420A4000E0082291
S1138E80009FF9188C4667450CD001982E21D040DC
S1138E90061C203EF6B25A2E00D8C1B23970083AE8
S1138EA00137F0E7009AD218029B0092013B02932B
S1138EB0002B03D00399002900D061E7009A0D2309
S1138EC013700A2353700023937008A800F018FF4E
S1138ED045E70023D356002B00D17EE2101C00F09E
S1138EE074FD051C112C01D0232C01D1B24800E0E3
S1138EF0B24800F005FF06A8FFF76FFA069B1A7840
S1138F00002A00D169E220218A4352B204214C2A6A
S1138F1002D0572A04D10221A94A0133116005E085
S1138F20422A04D1A64A012111605B18069306A8BF
S1138F30FFF753FA069800F048FD089006A8FFF7DB
S1138F404CFA112C02D00123232C08D106980022BC
S1138F5082560123002A02D000F053FD031C223C58
S1138F60E4B200260122A24276411C1C002C00DC43
S1138F7033E2934F3A68022A0BD0042A14D0012A10
S1138F8019D1089B002E02D007A90B7006E02B70A4
S1138F9011E0089B002E05D007A90B80281C02F0C5
S1138FA09FFB08E02B8006E0002E02D0281C08A9B5
S1138FB0F5E7089929603B68013CED18D6E70023E2
S1138FC0D356002B00D108E2101C00F0FEFC041C58
S1138FD006A8FFF702FA06980022825600218A4268
S1138FE002D000F0F2FC011C201C02F05FFB051E05
S1138FF001D17448F3E17448EDE1002909D0032953
S113900000D0EAE1714B101C1C6800F0FAFC2081CE
S1139010E3E16F4D2B88042B05D16E4800F070FE00
S113902010232B8004E06C4B081C1980FEF7FCFF16
S1139030251CE3E10892072900D9CEE1081C02F0BF
S113904037FF04244148134D523808A8FFF79DF90F
S1139050041C08A8FFF799F907A908700122201C2D
S113906001F004FC5D48B6E108A8FFF78EF9041C82
S113907008A8FFF78AF907A9087059480122044390
S1139080A0B201F0F3FB5748A5E108A807ACFFF72D
S11390907CF9211C012201F00AFC002807DB52485C
S11390A000F02EFE2078812100F03BFE95E14F4830
S11390B091E1464B402218684D4B196800F0CCFCF6
S11390C04C4888E1FEF7A4FF0020FFF777FA4A48EE
S11390D081E1012001F003FC48487CE1022001F019
S11390E0FEFB474877E10020FFF768FA454872E144
S11390F0162900D971E1081C02F0E4FE1700900063
S11391002A004000AE006F016F016F016F016F0113
S11391106F016F016F016F016F016F016F01CC006F
S11391206F016F016F013F013F01284B00241D684F
S113913007206043344B311C181800F00CFE002843
S113914001D12C732CE101340C2CF1D12F4842E1D4
S11391500023D356372B05D11C4B01221B685968B9
S11391600A4307E0382B07D1184B01221B685968C2
S113917091430A1C5A6013E125482CE1134B002447
S11391801D6805206043234B311C181800F0E3FDD3
S113919000280CD16A6806239A43131C002C04D0BF
S11391A0012C00D015E102224FE004224DE00134ED
S11391B0032CE6D118480EE11CC4000023C40000AF
S11391C0C4F0FF1F2BC4000034C40000E8F0FF1FEC
S11391D0F6F0FF1F44C400009EF1FF1F50C40000BE
S11391E00080FFFF62C400007AC400008FC4000046
S11391F0E0F0FF1FB1C40000D2C40000F2C40000BC
S11392000DC500002AC500000CC10000EAC500001D
S113921042C5000018D0000003C60000794B0024AA
S11392201D687948A300C018311C00F094FD002883
S11392300DD16968182399430B1C012C04D0022C0E
S113924000D0C6E0102200E008221343C1E001343C
S1139250032CE6D16D48BEE06A4B00241F686C48BD
S1139260E300C018311C00F076FD051E0DD07A68AD
S113927060239A43131C012C03D0022C03D1202217
S113928000E0402213437B608AE00134032CE6D1E2
S11392906048A4E0604800F033FD604800F030FD11
S11392A0584C21680B7B0B2B04D8072043435C48A4
S11392B0C01800E05B4800F023FD5B4D281C00F063
S11392C01FFD23682E1C5B68DA0701D5574800E0B0
S11392D0574800F015FD574800F012FD23685A68FE
S11392E00123910704D404231A40534253415B00E1
S11392F0052043435048C01800F002FD4F4800F0D9
S1139300FFFC236802205B68DA0601D41807C00F4B
S11393103D4B8000181800F0F3FC494800F0F0FCC5
S1139320236801255B68590602D49D06ED0F6D0084
S1139330444800F0E5FC3648EB00C01800F0E0FCBF
S1139340301C00F0DDFC002D47D03F4800F0D8FC75
S1139350236800213633187800F0DAFC3B4D281CD2
S113936000F0CEFC3A4800F0CBFC236800213733F0
S1139370187800F0CDFC281C2DE0101C00F041FBF7
S1139380C0B2632803D8002802D1012000E0632082
S11393901C4B1B68152C01D1363300E03733187091
S11393A00420FEF7DBFE18E0081C111CFFF73CF953
S11393B013E0062911D12748111C00F0CCFC051E2E
S11393C016D02548311C00F0C6FC051E0AD02348DF
S11393D001E06B60E4E700F093FC00250EE000F090
S11393E08FFC0BE0074B40211B685A898A4304E039
S11393F0044B40211B685A890A435A81281C13B024
S1139400F0BDC046E8F0FF1F32CE000016C60000D3
S113941030D000002CC600005AC5000073C50000FF
S11394200CC100007BC5000041C4000084C50000DD
S113943086C5000088C5000018D000000CC60000D6
S113944090C500009FC50000ADC50000B9C500006F
S1139450BDC50000C8C50000CFC50000D7C50000C9
S1139460F0B585B003910021071C02920191039984
S1139470002900D1F8E03B787D4C082B0CD17D4BC2
S11394801A78002A05D07C48013A01301A7000F09D
S113949037FC00232370E2E01B2B04D05B2B05D1A7
S11394A022781B2A02D123700137D8E022785B2A64
S11394B04BD1181C4138032847D802F0F9FC10108E
S11394C009026C4B1A78002A00D1C8E0013AC5E0C1
S11394D0684B1A78272A00D9C1E00132BEE0674CF4
S11394E028202268664E5043301800F059FC3B781F
S11394F0051C412B08D12368002B01D1032300E074
S1139500013B23605F4806E023680133032B00DD41
S113951000235D48236000F0F3FB002D04D05B487A
S113952000F0EEFB013DF8E7574800F0E9FB206846
S113953028256843301800F0E3FB20684543701980
S113954000F02EFC4B4B187089E00A2B00D186E00A
S1139550002B00D183E04749484C0A78216828252C
S11395606943474E89188B553B780D2B6AD10A23E2
S113957002988B55FEF7D6FD23683E4A5D43137867
S1139580434A0C2012784349424301337519545815
S1139590DBB28A185679EA180021013A117002994F
S11395A0002905D13C4A1288002A39D0510537D404
S11395B0002B32D0281C002E19D02168FEF7CDFED6
S11395C0013E0190002810D0344800F099FB207A25
S11395D0617A019AFFF756FA002802D1304800F068
S11395E08FFB029A002A1BD112E00C34E2E72D49CA
S11395F0FEF7B3FE021E10D004200921FFF742FA41
S1139600002802D1264800F07BFB029B002B07D1E7
S1139610214B1888FEF708FD02E0234800F070FB98
S1139620FEF792FD134B00221A70144B1968013196
S1139630032903DC19600121019106E01A6001226B
S1139640019202E00B4B01321A70094B00221A708E
S1139650084B01371A78272A01D927221A70039B4D
S1139660013B9BB2039302E7019805B0F0BDC046ED
S1139670F4F0FF1F9CF1FF1F51D00000F0F0FF1F1A
S1139680FCF0FF1F45C6000078C200001AC40000A9
S1139690A8F1FF1F9CCD0000A0F1FF1F41C40000F2
S11396A002C4000049C60000FEC3000013B5441EF6
S11396B0E4B21423634304480068C318187C00947C
S11396C05C680323A04716BDACF1FF1F08B5044B2B
S11396D018701423584300F093FB024B186008BD24
S11396E0A9F1FF1FACF1FF1F37B5031C0D1C0020AF
S11396F0FF2B0DD0013BDBB214245C430549096800
S11397000C19207C0093111C64682A1C0223A047B6
S11397103EBDC046ACF1FF1F13B5441EE4B2142392
S1139720634304480068C318187C00945C680423ED
S1139730A04716BDACF1FF1F421ED2B2142313B5CD
S1139740534305490968CB18187C002100925C68D2
S11397500A1C0523A04716BDACF1FF1F30B50A4B08
S11397600A4A1B6814780022A2420BD05D680132B9
S1139770854204D11D7C8D4201D1D0B203E0D2B226
S11397801433F1E7002030BDACF1FF1FA9F1FF1F36
S1139790F0B5061C85B0101C019102920393FFF7EB
S11397A0DDFF011E01D000203AE0FFF7D7FF071EBE
S11397B0F9D0142545431B4B143D1B685D193388B0
S11397C0002B13D0039800F01BFB041CA8600DD0E1
S11397D03388181C009300F013FB0028E3D0009B8F
S11397E020606060A060C018E060E3827388002B92
S11397F011D0039800F004FB041CE8600BD07688B9
S1139800301C00F0FDFA0028CDD020606060A0601C
S11398108019E060E682029B381C6B60019B2B740C
S113982005B0F0BDACF1FF1F07B500280ED0002134
S113983003280FD1108901AB126818805980117860
S1139840181C054A1823FFF7A3FF04E0101C00F0BE
S1139850BFFE00E0081C0EBDDD9A00002023F7B512
S11398600E1C141C194203D0137008239E430134A8
S1139870730706D5002804DA2D23237047420134E8
S113988000E0071C00232E4D0093002F36D0BD426C
S113989013D9281C0A2102F01FFB009B051C002B76
S11398A003D10128F3D1730601D5302302E0330735
S11398B0EDD5202323700134E9E7002D01D00123E5
S11398C00093291C381C02F007FB631C0193031C42
S11398D0C0B26843303323703F1A0A21281C02F0B7
S11398E0FBFA019C051CD0E7002B0DD0281C0A2193
S11398F002F0F2FA30232370051C0134201C009B73
S1139900002DF1D1002B0DD1330703D52023601C8A
S1139910237007E0730602D53023601C23703023C4
S11399200370013073B2002B04DA0D2303700A2391
S11399304370023010231E4000D10670FEBDC046A5
S113994000CA9A3BF7B520230090194201D0137046
S11399500132080704D53023137078235370023280
S113996040230B409C46CBB21026019307230E40A4
S113997019400F1C042900D904277F00FFB2141CCE
S11399803B1C013BDBB2FF2B11D000989D00E8404B
S11399900F21051C0D40291C3031392904D960469A
S11399A02731002800D0203921700134E9E70199DA
S11399B0D0194BB2002B04DA0D2303700A23437031
S11399C00230002E00D10670FEBD10B5031C00222B
S11399D09A56202A01D10133F9E700201A7851B2AE
S11399E02F290DDDD2B20101101C3038C0B2013371
S11399F0092803D9101C57380F2420400843EDE7E9
S1139A0010BD10B500220378191C3039092906D974
S1139A10002B17D02D2B00D101220130F3E70023B6
S1139A2001780C1C303C092C07D85C00303CDB006E
S1139A30E31849B201305B18F2E7181C002A02D07F
S1139A40584200E0181C10BD031C8218934202D037
S1139A5019700133FAE7704710B50023934203D01D
S1139A60CC5CC4540133F9E710BDF7B5038A041C78
S1139A700E1C4768151C9A4200D91D1CADB2002D5E
S1139A8028D0E3687A1962609A4215D3DB1B9BB233
S1139A902268E91A009353186360019101F04AFCAB
S1139AA0002E12D0391C009A301CFFF7D5FF009B02
S1139AB02168F018019A06E001F03CFC002E04D065
S1139AC0301C391C2A1CFFF7C7FF01F02BFC238A2A
S1139AD05B1B238201F02EFC281CFEBDF7B51D1C68
S1139AE008AB1B78171C14225A43164E0191316897
S1139AF000928B189C6801F015FC052D09D0062DE9
S1139B0009D0042D16D1201C01993A1CFFF7ADFF92
S1139B1016E0258A11E0012F03D13368009A9B18BF
S1139B20DC68002C08D02368258AA36063600023C6
S1139B30238202E0002500E0251C01F0FBFB281C29
S1139B40FEBDC046ACF1FF1FF7B5041C151C0F1C6D
S1139B5001F0E8FB218A628AE38A88184019984256
S1139B6002DD5D1AAD1AADB2A168AA186282019134
S1139B704A19E168A2602E1C8A4205D3D31A2268CE
S1139B80A3609B1AEE1AB6B201F0D4FB0198391CFB
S1139B90321CFFF761FFB54204D0B919AA1B206833
S1139BA0FFF75AFF01F0BEFB638AA28AAB4206D1DB
S1139BB0238AEB189A1800232282A38202E0AA18AF
S1139BC0A2825B1B638201F0B5FB281CFEBD000072
S1139BD0F7B5041C0191002936D1027843780D1C95
S1139BE09A4261D101F09EFBA178304B3048197044
S1139BF0FFF7B4FD2F49087000280ED014225043FB
S1139C002D4B1B6818181438836820791A8A561D3E
S1139C103618D88A864203DD0D7001F08BFB43E0D1
S1139C2006321A82A11D8C420CD09A68501C98608E
S1139C30207810709868DA68904201D318689860A8
S1139C400134F0E706252FE01A4B1E78002E0DD1C3
S1139C5002784378351C9A4226D187781448391CF7
S1139C60FFF77CFDFFB2061E06D11DE00F4A1778F0
S1139C7000221A7001F05EFB14220F4B56431B683E
S1139C809E19E378143EB068032B04D1C58A038A75
S1139C90ED1AADB208E0211C019AFFF755FF04212B
S1139CA0051C78B200F030FA281CFEBDABF1FF1F92
S1139CB0DD9A0000AAF1FF1FACF1FF1F08B5031ED7
S1139CC004D1081C111CFFF783FF05E00020FF2BC3
S1139CD002D0181CFFF7EAFC08BD38B5041C031CAD
S1139CE01A1B0133581E057892B2002DF8D1281C96
S1139CF0002A03D0081C211CFFF7E0FF38BD000038
S1139D0008B5024B1978FFF7E8FF08BDCCF0FF1F38
S1139D101FB56A46FFF7A2FD6846FFF7F1FF05B0DD
S1139D2000BD1FB56A46FFF70DFE6846FFF7E8FF62
S1139D3005B000BD07B5031C002083420AD06A4663
S1139D401070507093701171012368460521D3700F
S1139D50FFF73EFF0EBD0378002B0FD000228A567A
S1139D605BB2934207D0D80FD1179A424841404280
S1139D700123184307E001300131ECE700200856C5
S1139D80431E98414042704710B5031C0C78181CC0
S1139D901C700A78013352B20131002AF6D110BD89
S1139DA0021C031C981A0133591E097849B2002970
S1139DB0F8D170470E4B13B500221A800D4B0E4A92
S1139DC019600E4B147819601A1C0378A34203D04F
S1139DD0002B0CD00430F8E74388C91811606B4697
S1139DE00733994203D855230B700131F7E713BDAC
S1139DF0B4F1FF1FB0F1FF1FD2F0FF1FB8F1FF1F36
S1139E00F8B50E4F0E4E3B683488051C1C1903230D
S1139E101C4201D09C4304340A4A631912689A42D2
S1139E200AD92A1C201C0021FFF70EFE3B68201CC7
S1139E30E31AED18358000E00020F8BDB0F1FF1FF3
S1139E40B4F1FF1FB8F1FF1F084B10B51A68011CCD
S1139E50131C981A01331C7880B2552CF9D00028B1
S1139E6000D11A1C024B9A1A0A8010BDB8F1FF1FC8
S1139E70F02F0000034B1868034B1B68C01A80B214
S1139E807047C046B8F1FF1FB0F1FF1F044B1868BC
S1139E90044B1B68C01A044B1B88C01A80B270475D
S1139EA0B8F1FF1FB0F1FF1FB4F1FF1FF0B585B08B
S1139EB00392564F564A002313603B60554B029061
S1139EC01B780C1C2678002E44D09E423BD1231CC8
S1139ED0E51A00260134A657EDB2002EF8D114205D
S1139EE068430430FFF78CFFEB43E31838600193B9
S1139EF0371C019C6278002A23D0029B1968002930
S1139F001BD00C78A24216D15A68016042601A89AB
S1139F100281002A01D00136F6B2598941819A8919
S1139F2082819B7BC373002901D1002A01D00137B0
S1139F30FFB2143001E01033E0E7019B01330193D9
S1139F40D7E7026008E001340022A256002AFAD1C1
S1139F500134B7E7371C351C2C4C2368002B49D03F
S1139F60002F2CD00C207843043080B2FFF748FF38
S1139F70274A2368106094461A68002A1AD05A891E
S1139F80002A07D024498A4201D100225A815A89E1
S1139F90426003E09989002901D0416001224168AF
S1139FA0002901D001214172002A01D003600C3044
S1139FB01433E1E70C235F436346C01B1860039925
S1139FC07018C0B2FFF782FB002E13D024682268F9
S1139FD0002A0FD02389002B0AD003200121221C40
S1139FE0FFF722FC002801D0A07301E0FF23A37334
S1139FF01434ECE7094801F085F9094B00221A6092
S113A00001F04AFA281C05B0F0BDC046BCF1FF1FA0
S113A010C8F1FF1FD2F0FF1FFFFF0000C0F1FF1FB8
S113A020C4F1FF1F054A06481188CB07DB1703401C
S113A03049084B4098B210807047C046C0F1FF1FDA
S113A04000B4FFFF184B37B51C682368002B29D0D8
S113A050E27B0D231A4223D001F064F9A389002B7B
S113A06002D1E37BD90716D4237C002B0ED0002524
S113A0706A46157055702168281C0A7869468A70EA
S113A0800522CD700B71FFF719FE2574E27B0A23BC
S113A090134000D1E37301F04DF9201C626890472E
S113A0A01434D2E737BDC046BCF1FF1F38B50C4BA2
S113A0B0051C1C6801F036F92368002B0DD0E17BE8
S113A0C00D22114207D01B785BB2AB4203D001F0E2
S113A0D031F9012002E01434EEE7181C38BDC04603
S113A0E0BCF1FF1F074B1B681A68002A07D01278BF
S113A0F052B2824201D1D87B02E01433F4E78020CB
S113A1007047C046BCF1FF1F38B5174B1C68236865
S113A110002B27D01B785BB2834221D1002918D1B0
S113A120124B1D68002D14D02B68002B11D09C42BB
S113A1300DD101F0F7F8A389002B03D00C4A126863
S113A1409B186B600023E37301F0F4F80AE00C350C
S113A150EAE74A0702D5E37B1A0703D4E17301E077
S113A1601434D4E738BDC046BCF1FF1FC8F1FF1F4B
S113A170C4F1FF1FF8B5194B0E1C1C68171C002CEA
S113A1802BD0174B1D682B68002B26D01B785BB295
S113A190834220D12368002B1FD09D4219D101F0A6
S113A1A0C1F8EB7B02229343EB732772002F04D197
S113A1B0AE81002E04D1667208E0002E00D1012683
S113A1C0084B1B68F61801236660637201F0B2F84D
S113A1D003E00C34DEE71435D5E7F8BDC8F1FF1F02
S113A1E0BCF1FF1FC4F1FF1F38B5114B1D68002DD2
S113A1F01DD0104B1C682368002B18D01B785BB251
S113A200834212D12B68002B11D09C420BD101F058
S113A21089F800232B726B72E37B02221343E373EE
S113A22001F088F803E00C35ECE71434E3E738BDBB
S113A230C8F1FF1FBCF1FF1F134A144B11681B68C0
S113A240013110B5101C1160002B1CD01A68002AB3
S113A25019D0597A002914D001685C68A14210D140
S113A260D17B8C0705D40C0701D40421D173197A4E
S113A27011749289002A03D059688A185A6000E040
S113A2805A720C33E2E710BDC4F1FF1FC8F1FF1F7F
S113A290F0B50D1C2C352B7885B0061C0C1C9A07C8
S113A2A00FD01121DA0700D4132101F033F9C0B221
S113A2B0002861D12B7803229343402213432B704F
S113A2C05AE020271F4054D1088B002803D1402294
S113A2D093432B704DE0CA681178A26A520516D5D3
S113A2E00422134202D093432B7010E0221C2E321E
S113A2F012780192914205D02D22125D8A4206D134
S113A300012804D004210B4301992B700127301C30
S113A31001F000F923684022013323602B781343B2
S113A3202B70002F28D1E36862690133E360934204
S113A33001D3A368E360228B104B013AB600F358B3
S113A34092B222832F34998C2378002B14D08A4222
S113A35012D86A46937201230025D372DD23157245
S113A36055721373281C02A90522FFF7A7FC257058
S113A37002E0301C01F0EAF805B0F0BDD8F1FF1F8F
S113A380F7B5019308AB071C0D1C141C1E7800F0D4
S113A390C9FF01980238082800D9F7E001F088FDC8
S113A3A0054A713CCAF6F6F6A10014237A4A5E43C4
S113A3B012689319E90401D5DE6800E09E68002C58
S113A3C028D0E20703D5381C01F0FAF804E0A3070B
S113A3D002D5381C01F018F9610703D5381C01F0C7
S113A3E0C1F804E0220702D5381C01F0DFF8B36A93
S113A3F0E10603D580225201134303E0A20602D5ED
S113A400664A1340B362630604D57F231D40331CA0
S113A4102F331D70358DBAE0142256435E4B604ACB
S113A4201B689E19B3689C6A144201D01D8CAEE06F
S113A4301D8BACE01422584B56431B689E19F668DA
S113A440002D07D1F28B338BD31A9DB2A34200DBCC
S113A4509DE09BE000F06EFF301C291C221C08309C
S113A460FFF772FB051C00F05DFF331C2C331A78D8
S113A47060231A4200D08AE0381C311CFFF708FF21
S113A48085E014237343444901930968221CCB18C3
S113A4909E68291C301C0830FFF7E7FAB36A602273
S113A4A0051C134275D0321C2C3211781020014245
S113A4B06FD0348BA446B48CA4456AD88143117000
S113A4C0990666D5344C01202668019C3619F1683A
S113A4D00B1C2C331A7802431A70381CFFF7D8FE71
S113A4E057E02D4A1423012C08D95E431368023C1B
S113A4F09E19F368A4B2002D13D106E05E431268DE
S113A5009619B368002D0CD107E0012C05D91D6004
S113A5105D60B3681D605D6039E0A4000025E5500E
S113A52035E0A4001C190023E25CEA540133042B37
S113A530FAD12BE0184D1423002C04D05E432A6872
S113A5409619F3681BE05E43296810248A199368FE
S113A550191C2C310878204211D0A0430870D1680E
S113A5608A6A920608D50B1C2C331A780120024300
S113A5701A70381CFFF78CFE2B689E19B3689A6812
S113A58000251A61DA601D831D8400E0002500F0B7
S113A590D1FE281CFEBDC046ACF1FF1FFFEFFFFF3C
S113A5A08080000038B5051C3020FFF729FC041E0C
S113A5B001D100200BE0281CFFF722FCA06000283A
S113A5C0F7D043192061E0606361E583201C38BD46
S113A5D0F7B53E4E0091017A041C301CFFF7BEF81B
S113A5E0051C071C002D03D0009A520707D46BE00A
S113A5F0291CFFF7B3F8051C381C002D64D0142760
S113A6006F43334B143F1B68DF19009B7E609B072D
S113A61007D5E088267AFFF7C5FF2E4AB600905189
S113A620F860009B2C4EDB0706D5A088FFF7BAFF25
S113A630237AB8609B00F050237A264A9B00D358B3
S113A640002B0ED0226864219A62237A214A9B004F
S113A650D358E0880093A37B584301F08BFC009B04
S113A6609884237A9B00F358002B26D0227B2F3327
S113A6701A70237AA288607B9B00F35850436421AC
S113A6800092019301F076FC019B009A5884237A8E
S113A690A07B9B00F35850436421019301F06AFCB2
S113A6A0019B22689884237A9B00F3589A62237A48
S113A6B0A27A9B00F3582E331A70237A211C3B7420
S113A6C0207A00F0ABFF281CFEBDC04681A3000029
S113A6D0ACF1FF1FD8F1FF1FCCF1FF1FF7B55B4AA8
S113A6E08B009C585A4A80279D58A36A3F01061C38
S113A6F001911F4014D0221C2C32117804200F1C0D
S113A7000740BC4603D081431170002710E0271C8A
S113A7102E373F78B74202D10143117094E0674667
S113A7201A0605D5221C2D321778BF1B7A425741D1
S113A7302022134218D0132E08D12B1C2C33197845
S113A7400A431A706B6801336B607DE0112E0BD1E4
S113A7502B1C2C331978114276D09143197001982F
S113A760291CFFF795FD6FE0226801322260D904AD
S113A7701AD52A8BEB8B9A420CD82A6916702B694E
S113A780696901332B618B4201D3AA682A612B8B3F
S113A79001332B832B1C2C331A7860231A4203D1E8
S113A7A00198291CFFF774FD238BE28B002F32D113
S113A7B09A420BD90133238323691E702369676985
S113A7C001332361BB4201D3A1682161A36A6022E2
S113A7D013421BD0261C2C363278D70616D4218B74
S113A7E0628C914212D3990609D52B1C2C331A780A
S113A7F002210A431A700198291CFFF749FD337896
S113A800102213433370636801336360114BA26AEF
S113A8101A4211D018E0218C013121849A420BD9BB
S113A8200133238323691E7023696769013323611C
S113A830BB4201D3A16821612F342078002803D0C2
S113A84040B20421FFF760FCF7BDC046CCF1FF1F06
S113A850D8F1FF1F8080000008B5034B8200D15857
S113A860FFF716FD08BDC046D8F1FF1F70B5041CE4
S113A87001200E1C151C00F085FF002807D100F0F4
S113A88081FF002800D1412003235840C0B223B2E5
S113A890002B05DA80235B421843C0B203235840DF
S113A8A06404321C2B1C610C00F0B2FF70BD03B2B7
S113A8B070B5041C0E1C151C0120002B02DA640464
S113A8C0640C002000F05EFF002805D0211C321C1F
S113A8D02B1C00F081FF01E00120404270BD08B54F
S113A8E0022804D003280ED0012817D10CE0002040
S113A8F000F048FF002811D080235B421843002158
S113A900C0B20A1C06E0002000F03CFF002805D07D
S113A91001210022131C00F07BFF01E001204042D2
S113A92008BD08B500F0D8FD08BD00000B4B30B5DC
S113A93000221C1C00215956002908D05988814244
S113A94005D8002A02D055888D4200D91A1C211C32
S113A95006333C318B42EDD1101C30BDE6F1FF1FB4
S113A960084B10B51C1C00229A56002A04D08342BE
S113A97002D05A88521A5A80221C06333C3293421F
S113A980F1D110BDE6F1FF1FF0B5807B89B00190D5
S113A990019802A90522FEF7BFFE002837D06B46B6
S113A9A0DE7A002EF4D104AD1A4F2E706E70EE7064
S113A9B0381CFFF7BBFF041E13D0174B67881B8896
S113A9C0BB4202D206AE73800DE023780020AB7048
S113A9D02379291C2B7105222070FFF76FF9261C9F
S113A9E0E6E7002E05D07188002902D0301CFFF75D
S113A9F0B7FF0848FFF79AFF041EC9D04188012217
S113AA007020FFF7B7FB6288034B1A80C0E709B0D8
S113AA10F0BDC046FFFF0000E4F1FF1F08B5612050
S113AA20B721FFF787F908BDF8B53D4B3D4E1A68CD
S113AA30041C01321A6033780D1C0133DBB233700D
S113AA403B2B4DD9384F3B780133DBB23B703B2B6A
S113AA5039D9364B1A780132D2B2172A01D81A7072
S113AA6024E000221A70324A324811780378013106
S113AA70C9B211700133DBB2062B01D9073BFAE7E7
S113AA8003701D2907D12C4B1978022903D1012108
S113AA90117003221A702A0708D5E368002B05D029
S113AAA000F040FCE268904700F044FCAB0608D597
S113AAB06269002A05D000F035FC6369984700F00C
S113AAC039FC00233B70AA0708D56368002B05D026
S113AAD000F028FC6268904700F02CFC00233370DF
S113AAE0EB0508D5A268002A05D000F01BFCA3687A
S113AAF0984700F01FFCAA0508D52368002B05D051
S113AB0000F010FC2268904700F014FC2369002B2D
S113AB1005D000F007FC2369984700F00BFCF8BD52
S113AB2024F2FF1F29F2FF1F2AF2FF1F28F2FF1F42
S113AB30CEF0FF1FCDF0FF1FCFF0FF1F0D4B1B7892
S113AB40C3720D4B1B8883800C4B1B7883710C4B99
S113AB501B78C3710B4B1B7803720B4B1B7843722E
S113AB600A4B1B7883720A4B1B68036180230373AF
S113AB707047C04629F2FF1FD0F0FF1FCFF0FF1F20
S113AB80CEF0FF1FCDF0FF1F28F2FF1F2AF2FF1F98
S113AB9024F2FF1FF0B58C46002801D1414B196007
S113ABA0414C62460423611E89B28D070DD13F4D8D
S113ABB0AA420FD93E4E02339219DBB2062B02D8B9
S113ABC00134A4B2EFE7073BF7E73A4DAA4204D8B1
S113ABD0002500E00125002408E03749013352181C
S113ABE0DBB2062BECD9073BFAE70224002D0CD08C
S113ABF0012C0AD1314EB24217D9314C1D331219EE
S113AC00DBB2062BF1D9073BFAE72E4E2E4F365D09
S113AC107743BA4209D9D21BF318DBB2062B01D908
S113AC20073BFAE70134E4B2E0E70134E4B2012778
S113AC30254DAA4209D9254D01375219FFB20133D6
S113AC40DBB2062BF4D9073BFAE70025204EB242CB
S113AC5004D9204E01359219EDB2F7E700263B2ABC
S113AC6003D901363C3AF6B2F9E7D2B2002809D04A
S113AC70818061468471C7710372C27286724572A3
S113AC8001610DE0144804701448077014480370FF
S113AC90144B1A70144B1E70144B1D70144B1980F6
S113ACA0F0BDC04624F2FF1FB30700000085E20197
S113ACB0007B1DFE8033E10180CC1EFE803B26001C
S113ACC080C4D9FF5ED000008051010080AEFEFF39
S113ACD00F0E0000F0F1FFFFCFF0FF1FCEF0FF1FBB
S113ACE0CDF0FF1F29F2FF1F2AF2FF1F28F2FF1FDA
S113ACF0D0F0FF1FF0B58BB005AD01900C1C281CE3
S113AD0000211422FEF7A0FE0199042910D10B237F
S113AD102B73002C0FD0281C00F0EEFD2A69002AAA
S113AD2009D1201C7949FFF72FF8001BC0B2EAE0D3
S113AD30281CFFF703FF019B07261E403AD0002C76
S113AD4034D006261E40221C002E12D00021E879A1
S113AD50FEF784FD2E270770421C4021A879FEF7D8
S113AD607DFD021C07700132A8880021FEF776FDE4
S113AD70021C01990523194219D0002E02D0202368
S113AD80137001324021687AFEF768FD3A26067096
S113AD90421C4021A87AFEF761FD021C06700132B4
S113ADA0E87A4021FEF75AFD021C00E0221C141B25
S113ADB0E0B2A8E0002C00D196E0019A102A0AD152
S113ADC00023E3562B2B0BD101340023E356202B15
S113ADD0FAD0012604E0019B302B01D1102101910E
S113ADE0201CFEF70EFEC2B2071C039223781A1C25
S113ADF0303A092A01D80134F8E7002102918B4244
S113AE000FD00134201CFEF7FCFDC0B20290237861
S113AE10303B092B01D80134F9E7331C5A1E934106
S113AE20F6180022A25600239A4208D00134201CAE
S113AE30FEF7E7FD321C511E8A4183B2B618019A0F
S113AE40102A10D12278111C3039092901D8013473
S113AE50F8E7211C202A06D14A780134303A092A1D
S113AE6001D830210191019A92060BD5029A0399D7
S113AE70AA71274AE971934202D8FA21C9005B18E2
S113AE80AB802DE0032E25D8301C01F011F8020808
S113AE900C15039A02996A72A972EB7220E02A696E
S113AEA0FFB2BF1806E03C23FFB25F432B6902994F
S113AEB0FF187F182F610FE0E1221201FFB2574300
S113AEC02A690299BF183C224A43DBB2BF18FB1817
S113AED02B6101E0002E03D0281C2969FFF75AFEDC
S113AEE0019A302A00D179E7019B102B04D1094B38
S113AEF0059306232B7302E0012205AB1A73281C69
S113AF0000F0FAFC00200BB0F0BDC0466AD000008F
S113AF10CF0700001DAA0000F0B587B00591818815
S113AF200422039135490023039C0326A14214D231
S113AF304C1C314207D1324D02325B19D2B2062A7F
S113AF4009D9073AFAE72F4F0132DB19D2B2062AA0
S113AF5001D9073AFAE7211CE6E70E4081794C1E35
S113AF60002C0BD0284D013C655D284FAA186F4377
S113AF70DB19D2B2062AF3D9073AFAE7002E09D12F
S113AF80022907D9214D01325B19D2B2062A01D90F
S113AF90073AFAE7C679771ED219D2B2062A01D93E
S113AFA0073AFAE7447A0194857A0495C47A019DB4
S113AFB0E12000014543AC46049D3C2068430290D7
S113AFC06044051911484743EF19F818059B002BF5
S113AFD012D00F4B039D019F1D800E4B19700E4B19
S113AFE004991E700D4B1F700D4B19700D4B1C7086
S113AFF00D4B1A700D4B186007B0F0BDB20700007E
S113B0000085E2018033E1015ED00000805101003F
S113B010D0F0FF1FCFF0FF1FCEF0FF1F28F2FF1F5D
S113B0202AF2FF1F29F2FF1FCDF0FF1F24F2FF1F9A
S113B03010B586B0041C422301A80373019400F0E8
S113B0405BFC021E012A05D1034B6B2014211C60FA
S113B050FFF790F806B010BD2CF2FF1F10B5847BEB
S113B06088B0201C69460522FEF756FB00280BD049
S113B0706A46D378002BF4D11379012BF1D1034B19
S113B0801868FFF7D5FFECE708B010BD2CF2FF1FDE
S113B090F8B5204B051C1421186800F01DFF1E494B
S113B0A0071C00F019FF2A1C0021041CFEF7D6FB24
S113B0B0194D44216C434170612181707921C17023
S113B0C073213D1B20220171E1210270861D427112
S113B0D00901281C00F000FF321C0021041CFEF7AB
S113B0E0BDFBE1231B015C433A262C1B471C067065
S113B0F03C21201C00F0F0FE3A1C4021051CFEF708
S113B100ADFB0670421C3C2045434021601BFEF70A
S113B110A5FBF8BDC4F1FF1F8051010008B56C20E8
S113B120FEF7C4FF002801D100F0E0FC08BD704721
S113B1307047704770477047704770477047704753
S113B14070B5164C164D23782A78DBB21A40910656
S113B1500CD5144A144E9078337802211840FFF726
S113B160BDFA2378DBB21A0700D532782A783F215A
S113B1708A431A4202D00220FFF76EFB2A7840234A
S113B1801A420AD02178194207D09A43044B1A7004
S113B190064B042219689143196070BD04C006402F
S113B1A003C00640A8F2FF1F07C0064068F2FF1F55
S113B1B070B5164C164D23782A78DBB21A409106E6
S113B1C00CD5144A144E5078337801211840FFF7F7
S113B1D085FA2378DBB21A0700D532782A783F2122
S113B1E08A431A4202D00120FFF736FB2A78402313
S113B1F01A420AD02178194207D09A43044B1A7094
S113B200064B022219689143196070BD04B00640D0
S113B21003B00640A8F2FF1F07B0064068F2FF1F04
S113B22070B5164C164D23782A78DBB21A40910675
S113B2300CD5144A144E1078337800211840FFF7C7
S113B2404DFA2378DBB21A0700D532782A783F21E9
S113B2508A431A4202D00020FFF7FEFA2A784023DC
S113B2601A420AD02178194207D09A43044B1A7023
S113B270064B012219689143196070BD04A0064071
S113B28003A00640A8F2FF1F07A0064068F2FF1FB4
S113B290154B10B51A68802001321A60134B144CF8
S113B2A01968014319602368590706D511490968CB
S113B2B08A4202D14200134323600F4A1368002BD1
S113B2C008D0013B1360002B04D1226880239B002B
S113B2D01343236021680948FFF7A6FB2168084B44
S113B2E00B40236010BDC046F82F002000D003405F
S113B2F064F2FF1F5CF2FF1F34F2FF1F3CF2FF1FDA
S113B300FFFCFFFF054B10B51C682388002B00D100
S113B310034B0380FEF786FE208010BDACF2FF1FB6
S113B3207B12000072B6024B1A6801321A60704731
S113B33060F2FF1F034A1368013B1360002B00D126
S113B34062B6704760F2FF1F08B58022044B920476
S113B3501A60FFF7E7FFFEF76FFFFFF7EBFF08BD8B
S113B36004ED00E0314BF7B51C68002C14D1304CCF
S113B37001239C43251C3C35231C01952D4D1E881F
S113B3802F1BDE53019F0233BB42F7D1274C0135FB
S113B390294B256013241C70284C23785BB2002BA6
S113B3A0FADA257830231D4200D02370244D00237F
S113B3B02B70244B18709C46062801D00A2827D1EC
S113B3C00E0C214BF6B201271E702F700F0AFFB22C
S113B3D06446C9B227701A4E1A4D1970062817D13F
S113B3E0022131705178297011781970032131705C
S113B3F0D1782970917819700421317051792970AC
S113B4001179197005213170D179297092791A70E6
S113B410FFF788FF054D094E2B6808489847FFF74A
S113B42089FF307833231840FEBDC04638F2FF1F31
S113B430D4F0FF1F6CF2FF1F03000240050002401E
S113B4400100024009000240080002400E4B10B502
S113B4501B6884004033E2500C4A89018318C9B246
S113B4601970C317DB0E1B18094A5B119B009B184C
S113B470084A104004D520220138524210430130BA
S113B480012282401A6010BD08ED00E000E400E0F3
S113B49000E100E01F000080084A094BDA63094B11
S113B4A0094A1360094A1360094BC022196812063D
S113B4B00A431A60074B07221A60704749B3000019
S113B4C000F0FF1F7F841E0014E000E018E000E09D
S113B4D020ED00E010E000E008B5094B1B785BB2FA
S113B4E0002B08DAFFF71EFF064B074A1A80074AAB
S113B4F01A80FFF71FFF8022054B92041A6008BDD3
S113B5000020054002200540A6020000B480FFFF91
S113B5104C0000F810B50B4B8200D35801221C7963
S113B52064B2002C0CDA084C82402068024322608A
S113B5301A79D9718022D97852420A43DA700022EA
S113B540101C10BD70D1000068F2FF1F044B800076
S113B550C3587F22D9780A4040210A43DA707047E1
S113B56070D100000D4B820010B5011CD458012885
S113B5700AD0002804D002280BD10E20084A06E085
S113B5800C200221074A02E0074A0D200221FFF79E
S113B5905DFFE37808221343E37010BD70D100000F
S113B5A041B1000021B20000B1B10000034B8000A2
S113B5B0C3583722D9780A40DA70704770D1000036
S113B5C00D4B820010B5011CD45801280AD0002864
S113B5D004D002280BD10E20084A06E00C200221D8
S113B5E0074A02E0074A0D200221FFF72FFFE37804
S113B5F024221343E37010BD70D1000041B1000058
S113B60021B20000B1B10000034B8000C3582421D3
S113B610DA788A43DA70704770D100001F4B8200D9
S113B62030B5D35801280BD0002805D0022834D1D6
S113B63080241B4AE40306E08024194A640302E0E0
S113B6408024174AA40315682C431460CC7A412241
S113B6500B2C02D8134A6400A25AD404E40ED2B2CA
S113B6601C705A700A68104C0621D50709D57F252D
S113B6702554114010D0510701D503220AE00222BB
S113B68008E0FF252554114006D0540701D51322A4
S113B69000E012229A7000E0997030BD70D1000071
S113B6A0148004407CD00000A8F2FF1F38B5440A7F
S113B6B0451864020A20211C0022FFF753FE0028CB
S113B6C006D180232A1B9B009A4202D9E418F1E791
S113B6D0012038BD08B58021C900FFF7E7FF08BD88
S113B6E0F7B507230191161C204C002909D12268C3
S113B6F01A4201D1002038E09A43226008220092C5
S113B70004E0021C9A43184022600090009B082524
S113B710ED1AB54200D9351C154A009B0199D7187A
S113B720381C2A1CFEF798F9019A114B52197F19FB
S113B73008330192761B9F4210D3062021680C4ADD
S113B740FFF710FE051E0FD1236809480833FF21B7
S113B75008222360FEF778F9009502E023685D195A
S113B7602560002ED2D1C5E70120FEBD30F2FF1FB7
S113B77054F2FF1F08B5031C081C191CFEF76CF9D2
S113B78008BD000030B5C42185B0051C49026846D7
S113B79010226B425D41FEF75FF90E4C009B6D4237
S113B7A02543A34202D1029BAB420FD0C621684677
S113B7B049021022FEF750F9009B0020A34206D153
S113B7C00298401B45426841400000E0012005B05A
S113B7D030BDC04655555555F8B5151C1E1C0228DC
S113B7E001D0C42400E0C62464021034C9000C193A
S113B7F0281CAA1992B283B29A4207D0471C211C72
S113B8000122FEF729F90834381CF2E70020F8BDBC
S113B810F0B585B00193002543B20F1C0092AB42F2
S113B82002DA7F2318400125410608D5C4204002CE
S113B830FFF750FFC6204002FFF74CFF02E0C6248A
S113B840022800D0C424019B6402002B11D1002DD6
S113B85009D0C4204002844201D1C6204002FFF72F
S113B86039FF002520E0201CFFF734FF002F1BD0F8
S113B8703BE0231C1033FF00FF1801235B42009EB2
S113B8800393019B0099CA1892B2B3B29A420BD0A7
S113B8903378174A381C134302A908220293083745
S113B8A0FFF71EFF0136ECE7211C02A80822FEF771
S113B8B0D3F8104E0299B14205D0201C02A90822E7
S113B8C00296FFF70DFF002D0FD1083402A8211CAA
S113B8D00822FEF7C1F8029BB34206D0054B201C98
S113B8E002A908220293FFF7FBFE002005B0F0BD79
S113B8F000FFFFFF55555555F8B5037B041CF02296
S113B900181C904301380A2800D992E000F0D0FABC
S113B91008063E2A2D30831B1F251800002522E02F
S113B920454D980606D521690020FFF733F92469AF
S113B9302C607EE0201C0121FFF7EEFA286078E0FD
S113B9403E4B19680AE0201CFFF7F8F871E0201C50
S113B9500021FFF7E1FA20616BE02169201CFFF769
S113B96019F966E00125013500E0002501350BE0F9
S113B970334A042110682025884310601D402F4E4F
S113B98043D0216900253160013500E000250135EF
S113B990237B01272A4E7F2B04D93368AF40BB4356
S113B9A0336046E0274B20681A6803213A431A6043
S113B9B0254BAA00D050254A1420FFF747FD244BFD
S113B9C003211A78AF400A431A70224B9222920044
S113B9D031681A603D1C204B204A0D431A603560C3
S113B9E0237B5A0625D51E491E4B0888124A9842C5
S113B9F008D0002313601C4A13801C4A13601C4B9C
S113BA000B8016E011680020A9E7201C291CFFF711
S113BA1083FA3060B8E7637AE12212015A43A37AC9
S113BA203C214B43D218E37A0025D218114B1A60FB
S113BA30AEE70020F8BDC046F82F00205CF2FF1FDF
S113BA4064F2FF1F148004403CF2FF1F91B2000017
S113BA500040064004D0034000D00340C0870000EB
S113BA60F22F002035CA0000F02F0020F42F002010
S113BA7035CAFFFF34F2FF1F30B51A4C83001B197F
S113BA801C68D50701D50C4300E08C431C6080245E
S113BA900123640400280DD1080B0340880401D558
S113BAA002200343214201D0042003438C010FD51B
S113BAB008210CE00B401B018D0701D52020034316
S113BAC0214201D040200343880101D580210B434A
S113BAD00549940702D50D682B4301E0086803402B
S113BAE00B6030BD0890044014900440F8B5314B0D
S113BAF004211C68304A0C423FD0304800680028BA
S113BB0003D018688843011C36E01068C0020ED5C3
S113BB102B4840260578354305702A4D2F783E433F
S113BB202E700078C50702D518688843186010681D
S113BB3080020FD5244940250878284308702348FB
S113BB400678354305700978CD0703D519680420B4
S113BB5081431960106840020FD51D4940250878BB
S113BB60284308701B480678354305700978CD07CB
S113BB7003D5196804208143196030BF1C60106824
S113BB80C00204D50F4B4020197881431970116805
S113BB90890204D50D4B402019788143197013682C
S113BBA05A0204D50B4B40211A788A431A70FFF7C6
S113BBB0C1FBF8BD10ED00E01480044068F2FF1FE3
S113BBC005A0064000A0064005B0064000B00640AF
S113BBD005C0064000C0064008B56C20FEF782FA96
S113BBE00923021C00201A4207D0044B18680423BE
S113BBF00340584243410220C01A08BD10ED00E042
S113BC0010B5E023041C9C43012C07D0022C0DD05A
S113BC10002C10D16C20211CFEF776FA084B04216D
S113BC201A688A431A60002C05D108E0044B0421E9
S113BC301A680A431A606C200121FEF765FA10BDE8
S113BC4010ED00E0014A024B1A60FEE70400FA0519
S113BC500CED00E010B5124A12490023891A8B42F8
S113BC6004D01148C05CD0540133F8E70F49104A9E
S113BC70914204D10F4A10490023891A08E00F4861
S113BC800023801A8342F5D0CC5CD4540133F9E705
S113BC908B4204D0D018002404700133F8E710BD9F
S113BCA0C0F0FF1FE0F0FF1F7CD1000010800000F7
S113BCB010800000E0F0FF1FB0F2FF1F38C000004A
S113BCC0F8B5504D30212B684F4C8B432B602368C3
S113BCD001208B43021C2360FFF7CEFE4B4B202038
S113BCE01B684B4F03409C464A4E4B4B2A1C6546EF
S113BCF01F804A491E80002D0BD1494E41233370C9
S113BD004848494B65460380484B1D8080230B708F
S113BD1009E0434E002333700125424E6D423580C5
S113BD20424D2B8008701168414B80250B401360F5
S113BD30404BAD041A68291C2A431A6001200222D0
S113BD40FFF79AFE23680C221D433B4B25601A60C3
S113BD503A4BB4221A701A78D607FCD5384B1822FD
S113BD601A70384B1A78191CD006FAD40A78354B55
S113BD705506FBD5344A802149041160334A002119
S113BD801170197880220A431A70314B314A9A6033
S113BD90314ADA60314A1A61314A5A61314A9A6148
S113BDA0314A1A63314A9A63314ADA62314A324972
S113BDB0116032498A4201D00432F8E7304A1360F4
S113BDC0FFF748FFFF2108222E48FDF73DFE2E4BCA
S113BDD02E4A13602E4A13602E4B1A6805221A60ED
S113BDE0FCF7BAFA2C4A2D4B2D482E491A60FDF760
S113BDF0E1FF2D482D490322FEF758F8FEF722F9FA
S113BE00FCE7C04658F00F4054F00F4050F00F408C
S113BE10C5200000D928000002200540002005406C
S113BE20012005400420054007D0FFFF06200540FF
S113BE30FFFFFFFD40F00F40048004400050064027
S113BE40004006400440064024800440014006406F
S113BE5000F0FF1F3DB100002FB1000031B1000020
S113BE6033B1000035B1000037B1000039B1000032
S113BE703BB1000040F0FF1F3FB10000B0F0FF1FD6
S113BE8008ED00E054F2FF1FFFFFFF0014E000E0A4
S113BE9018E000E010E000E0FC2F0020ACF2FF1FEF
S113BEA094D00000B0F2FF1FF4D0000064D1000071
S113BEB002B4714649084900095C49008E4402BC39
S113BEC07047C04603B47146490840004900095A06
S113BED049008E4403BC7047002934D0012300225A
S113BEE010B488422CD301242407A14204D28142F5
S113BEF002D209011B01F8E7E400A14204D2814205
S113BF0002D249005B00F8E7884201D3401A1A4381
S113BF104C08A04202D3001B5C0822438C08A042B8
S113BF2002D3001B9C082243CC08A04202D3001B6E
S113BF30DC082243002803D01B0901D00909E3E7E8
S113BF40101C10BC7047002801D00020C04307B467
S113BF50024802A14018029003BDC046D900000067
S113BF600029F0D003B5FFF7B9FF0EBC4243891A8C
S113BF701847C046002941D010B4041C4C40A446C4
S113BF8001230022002900D54942002800D540425F
S113BF9088422CD301242407A14204D2814202D234
S113BFA009011B01F8E7E400A14204D2814202D254
S113BFB049005B00F8E7884201D3401A1A434C0851
S113BFC0A04202D3001B5C0822438C08A04202D387
S113BFD0001B9C082243CC08A04202D3001BDC08AF
S113BFE02243002803D01B0901D00909E3E7101CF0
S113BFF06446002C00D5404210BC7047002806D08F
S113C00003DB0020C043400801E08020000607B4A1
S113C010024802A14018029003BDC0461900000066
S113C0200029EBD003B5FFF7A7FF0EBC4243891AE2
S10BC0301847C0467047C046E2
S113C038210078002000000017005D600A0000005D
S113C0480041444D494E002020755461736B65725C
S113C058264B494E45544953000000000000000097
S113C068000000000000501403030000000000005A
S113C0780D0A0A48656C6C6F2C20776F726C642EFD
S113C0882E2E204B494E455449530D0A004F532038
S113C0984865617020757365203D20002066726FC5
S113C0A86D200052544320416C61726D20666972A0
S113C0B865640D0A00436F6D6D616E64206C696E72
S113C0C86520626C6F636B65640D0A00436F6E6E66
S113C0D8656374696F6E2074696D6564206F757427
S113C0E80D0A004C6F636B757000000001C70000F7
S113C0F804C700000012000014C7000019C700009C
S113C10802000000333030000000003630300000F8
S113C118000031323030000000323430300000008A
S113C1283438303000000039363030000000313403
S113C1383430300000313932303000003338343094
S113C1483000003537363030000031313532303088
S113C158003233303430300057444F470000000079
S113C16801C7000004C700000012000014C7000043
S113C17819C700000200000001C7000004C700003E
S113C1880012000042C700002CC700000000000095
S113C19814C7000019C7000002000000536F66743A
S113C1A8776172650000000001C7000004C7000041
S113C1B800120000D2CA0000DBCA0000050000001B
S113C1C8F0CA0000F9CA00000501000011CB000004
S113C1D81ACB0000050200002ECB000036CB00006D
S113C1E80503000051CB00005ACB000005040000F1
S113C1F87ACB000089CB000005150000A4CB000011
S113C208B2CB0000051600007AC70000CFCB0000AF
S113C2180511000099C700009EC70000030600002E
S113C22842C700002CC700000000000014C700002B
S113C23819C7000002000000436C6F636B206C6F29
S113C2487373000001C7000004C700000012000057
S113C25814C7000019C7000002000000536F667479
S113C268776172652076657273696F6E20000A0AB9
S113C2780D000A0D3D3D3D3D3D3D3D3D3D3D3D3DB2
S113C2883D3D3D3D3D3D3D0A0D000A0D5365726936
S113C298616C206E756D6265723A2000446576693A
S113C2A86365206964656E74696669636174696F3E
S113C2B86E3A20004E657720616C61726D2073655B
S113C2C8740D0A00416C61726D20636C656172655E
S113C2D8640D0A004E65772074696D652073657472
S113C2E80D0A004E65772064617465207365740DCA
S113C2F80A0030203D2052554E0031203D20574140
S113C30849540032203D2053544F5000205B616350
S113C318746976655D004C61737420726573657425
S113C328206361757365203D20000A0D5379737489
S113C338656D206D656D6F7279207573653A0A0DA8
S113C34800467265652068656170203D20000A0D0D
S113C358556E7573656420737461636B203D2000AA
S113C368202800290A0D000D0A54686520646576A2
S113C37869636520686173206265656E206F706506
S113C388726174696E6720666F722000426164206E
S113C398706F7274206E756D6265720D0A000D0AF5
S113C3A8506F727420646972656374696F6E3A20A1
S113C3B8004F55545055540D0A00494E5055540DCC
S113C3C80A00496E76616C696420706F72740D0A94
S113C3D800506F727420697320696E7075740D0A49
S113C3E800506F72742073746174653A2000310DC3
S113C3F80A00300D0A000D0A3F3F0D0A23004D655F
S113C4086D6F727920446973706C61790D0A00202C
S113C4182020200046696C6C0D0A00577269746507
S113C4280D0A004572617365640D0A0045726173F3
S113C43865206661696C6564210D0A000A0D4279FC
S113C44865204279650A0D000A0D506172616D65B7
S113C458746572207365740A0D000A0D54656D7055
S113C4682E20506172616D65746572207365740A5B
S113C4780D000A0D506172616D65746572207661F4
S113C4886C7565203D20000A0D4E6F2076616C693D
S113C4986420706172616D65746572732061766180
S113C4A8696C61626C650A0D000A0D4F72696769EF
S113C4B86E616C20706172616D657465727320724F
S113C4C86573746F7265640A0D000A0D46616374BE
S113C4D86F727920706172616D6574657273207210
S113C4E86573746F7265640A0D000A0D5061726198
S113C4F86D657465727320696E76616C69646174C4
S113C50865640A0D000A0D4E657720506172616DED
S113C51865746572732076616C6964617465640A14
S113C5280D000A0D436F6E66696775726174696FF1
S113C5386E2073617665640A0D00496E636F7272CA
S113C5486563742064617461206C656E6774680D3A
S113C5580A000D0A53657269616C20636F6E66691F
S113C5686775726174696F6E0D0A004261756420A3
S113C5783D2000696E76616C6964210037003800DB
S113C58820426974730D0A002073746F7020626905
S113C598742873290D0A00466C6F7720636F6E74D4
S113C5A8726F6C200048696768207761746572202F
S113C5B800250D0A004C6F7720776174657220009E
S113C5C8656E61626C650064697361626C65000D17
S113C5D80A496E76616C6964207377697463680DBF
S113C5E80A00496E636F72726563742073657269B9
S113C5F8616C2073706565640D0A00496E636F721F
S113C60872656374207061726974790D0A00496EE9
S113C618636F72726563742073746F7020626974D7
S113C628730D0A00496E636F727265637420666CD9
S113C6386F7720636F6E74726F6C0D0A000A0D0DAC
S113C648004D41430020202020204D61696E206D5B
S113C658656E7500204C414E20636F6E6669677580
S113C668726174696F6E0020202053657269616C71
S113C67820636F6E6669672E0020496E7075742F8B
S113C6884F7574707574206D656E75002020204197
S113C698646D696E2E206D656E75002020205374BC
S113C6A86174732E206D656E75002020202055530B
S113C6B842206D656E750020202020493243206D8C
S113C6C8656E750020204469736B20696E74657209
S113C6D866616365004654502F54454C4E455420BA
S113C6E8636F6D6D616E64730020202043414E209A
S113C6F8636F6D6D616E647300757000676F20748D
S113C7086F206D61696E206D656E75007175697451
S113C718004C6561766520636F6D6D616E64206D94
S113C7286F646500446973706C6179206D656E751A
S113C7382073706563696669632068656C70007549
S113C748705F74696D650053686F77206F706572E8
S113C7586174696E672074696D65006D656D6F72CB
S113C768790053686F77206D656D6F7279207573E2
S113C778650073686F775F636F6E666967005368F7
S113C7886F7720636F6E66696775726174696F6E1F
S113C7980073617665005361766520636F6E666920
S113C7A86775726174696F6E20746F20464C4153CB
S113C7B8480072656A656374005265736574206E17
S113C7C86F6E2D7361766564206368616E67657347
S113C7D800726573746F726500526573746F726565
S113C7E820666163746F72792073657474696E6707
S113C7F8730073686F775F74696D6500446973705B
S113C8086C617920646174652F74696D6500736562
S113C818745F74696D65005365742074696D65206F
S113C82868683A6D6D3A7373007365745F64617414
S113C838650053657420446174652064643A6D6DC1
S113C8483A797979790073686F775F616C61726D91
S113C85800446973706C617920616C61726D206445
S113C8682F74007365745F616C61726D0053657435
S113C87820616C61726D20286461746529282B29F4
S113C8885B74696D655D0064656C5F616C61726D94
S113C8980044656C65746520616C61726D00736831
S113C8A86F775F6C700053686F77206C6F772070B8
S113C8B86F776572206D6F646520616E64206F7098
S113C8C874696F6E73007365745F6C70005B6F706E
S113C8D874696F6E5D20536574206C6F7720706F78
S113C8E8776572206D6F64650072657365740052B4
S113C8F86573657420646576696365006C61737437
S113C9085F7273740052657365742063617573652F
S113C918006D64004D656D6F727920446973706CA5
S113C9286179205B616464726573735D205B3C6C40
S113C9383E7C3C773E7C3C623E5D205B6E756D5D63
S113C948006D6D004D656D6F7279204D6F64696679
S113C95879205B616464726573735D205B3C6C3E33
S113C9687C3C773E7C3C623E5D205B76616C5D007E
S113C9786D66004D656D6F72792046696C6C205B3D
S113C988616464726573735D205B3C6C3E7C3C77C8
S113C9983E7C3C623E5D205B76616C5D205B6E751F
S113C9A86D5D0073640053746F7261676520446938
S113C9B873706C6179207B6173206D647D00736D85
S113C9C80053746F72616765204D6F6469667920DE
S113C9D87B6173206D6D7D0073660053746F7261A3
S113C9E867652046696C6C207B6173206D667D00E9
S113C9F853746F72616765204572617365205B616A
S113CA086464726573735D205B6C656E2D6865780C
S113CA185D007365745F6464720053657420706F9D
S113CA2872742074797065205B312E2E345D205B1E
S113CA383C693E7C3C6F3E006765745F64647200C9
S113CA4847657420646174612064697265637469FC
S113CA586F6E205B312E2E345D00726561645F70E9
S113CA686F7274005265616420706F727420696E0D
S113CA78707574205B312E2E345D0077726974658D
S113CA885F706F72740053657420706F7274206FD6
S113CA987574707574205B312E2E345D205B302FD5
S113CAA8315D0054656D702074657374005361764C
S113CAB86520706F72742073657474696E67206181
S113CAC8732064656661756C74007365745F626174
S113CAD87564005365742073657269616C206261C2
S113CAE875642072617465007365745F73746F7024
S113CAF8005365742073746F7020626974732028FE
S113CB08312F312E352F3229007365745F626974B1
S113CB1873005365742064617461206269747320BE
S113CB2828372F3829007365745F70617200536564
S113CB38742070617269747920284556454E2F4FC8
S113CB4844442F4E4F4E4529007365745F666C6FDD
S113CB58770053657420666C6F7720636F6E747208
S113CB686F6C2028584F4E2F5254532F4E4F4E451A
S113CB7829007365745F686967685F7761746572B3
S113CB880053657420666C6F77207374616C6C2035
S113CB98282529205B312E2E39395D007365745F91
S113CBA86C6F775F77617465720053657420666C87
S113CBB86F77207265737461727420282529205B4D
S113CBC8312E2E39395D0053686F77207365726989
S113CBD8616C20636F6E66696775726174696F6EE4
S113CBE8003100436F6E666967757265204C414E6B
S113CBF820696E74657266616365003200436F6E06
S113CC086669677572652073657269616C20696EFF
S113CC1874657266616365003300476F20746F2022
S113CC28492F4F206D656E75003400476F20746F6F
S113CC382061646D696E697374726174696F6E20C2
S113CC486D656E75003500476F20746F206F7665CB
S113CC5872766965772F7374617469737469637321
S113CC68206D656E75003600476F20746F2055532C
S113CC7842206D656E7500476F20746F20493243FA
S113CC88206D656E7500476F20746F20757446417A
S113CC9854206469736B20696E7465726661636598
S113CCA80039004654502F54454C4E455420636C6B
S113CCB869656E7420636F6D6D616E6473006100E5
S113CCC801C7000004C700000012000019C90000D1
S113CCD81CC90000010F000049C900004CC900002C
S113CCE80110000078C900007BC900000111000090
S113CCF8ABC90000AEC9000001210000C6C900008C
S113CD08C9C9000001220000E0C90000E3C900000D
S113CD180123000077C70000F8C9000001250000BE
S113CD281ACA000022CA00000102000040CA00001A
S113CD3848CA0000010B000062CA00006CCA000067
S113CD480104000083CA00008ECA00000105000027
S113CD58B0CA0000ABCA0000014B000099C700002C
S113CD68B5CA0000010C000042C700002CC700002F
S113CD780000000014C7000019C7000002000000EA
S113CD887065726970686572616C206661696C753A
S113CD987265000070CF00000F0C00004DC6000043
S113CDA800D00000140200005CC60000B0C10000FE
S113CDB8160C00006FC60000C8CC00000F1000005D
S113CDC881C600008CCE00001111000094C600003A
S113CDD840CE000011050000A3C6000080C1000079
S113CDE80D030000B2C6000058CF00000D02000079
S113CDF8BFC600004CC200000D020000CCC60000F3
S113CE08F4C000000F020000DDC6000068C1000085
S113CE180F020000F1C60000486F73742064656255
S113CE287567676572003F3F3F0031000000312E8F
S113CE38350032000000000001C7000004C70000EC
S113CE480012000047C700004FC70000010A000095
S113CE5863C700006AC700000101000042C7000060
S113CE682CC700000000000014C7000019C7000008
S113CE7802000000556E646572766F6C74616765B4
S113CE880000000001C7000004C7000000120000F1
S113CE987AC7000086C700000602000099C7000090
S113CEA89EC7000003060000BAC70000C1C70000FF
S113CEB803070000D9C70000E1C70000030200000F
S113CEC8FAC7000004C80000060A000016C80000DB
S113CED81FC800000609000031C800003AC8000055
S113CEE8060800004EC8000059C80000060C0000DF
S113CEF86BC8000075C80000060B00008FC800004E
S113CF0899C80000060D0000A6C80000AEC80000BD
S113CF1801260000CEC80000D5C800000127000083
S113CF28F1C80000F7C800000100000004C90000AF
S113CF380DC900000120000042C700002CC70000F2
S113CF480000000014C7000019C700000200000018
S113CF5801C7000004C700000012000014C7000045
S113CF6819C7000002000000E9CB0000EBCB000069
S113CF780004000003CC000005CC000000050000FC
S113CF8820CC000022CC00000006000031CC0000B8
S113CF9833CC0000000700004DCC00004FCC00004B
S113CFA8000900006ECC000070CC0000000A0000EC
S113CFB884C500007FCC0000000E000086C5000078
S113CFC88ECC0000000F0000A9CC0000ABCC000000
S113CFD800100000C6CC0000F4C6000000110000D8
S113CFE842C700002CC700000000000014C700005E
S113CFF819C700000200000001C7000004C70000B0
S113D0080012000014C7000019C700000200000045
S113D0184F444400004556454E004E4F4E4500458A
S113D028787465726E616C004E4F4E4500000000C6
S113D0385254530000000000584F4E0000000000F6
S113D048506F7765722D6F6E000820080056312ED8
S113D058342E303132001F1C1F1E1F1E1F1F1E1F9F
S113D0681E1F4E6F20616C61726D20656E61626C6B
S113D07865640000471023081204090204018200B1
S113D08857004100210016000B0005000100002094
S113D0980000000048544D004A50470047494600E4
S113D0A8504E4700435353004A530042494E0054DC
S113D0B858540049434F00424D50003F3F3F0057EA
S113D0C8646F670061707000706572696F64006DE9
S113D0D861696E74656E616365006B656570657220
S113D0E8006C6F77506F776572000000C7D000003E
S113D0F823A900000000000004000100CCD00000B7
S113D108D58100004500020000000000D0D00000D6
S113D11889A900002500FFFF00000000D7D0000007
S113D128018500002500FFFF00000000E2D0000098
S113D1385DB000002500FFFF00000000E9D00000FA
S113D1481DB1000000000000000001000000000004
S113D1580000000000000000000000000157616D9D
S113D168706B6C000000000000A0064000B0064090
S107D17800C00640A9
S113D17CFF0000000100000001000000FF04010199
S113D18CB20701008021017001780906FCD57047B3
S90380106C
